:020000020000FC
:0200000015C029
:0200040018954D
:02000800189549
:02000C00189545
:02001000189541
:0200140018953D
:02001800189539
:02001C00189535
:02002000189531
:0200240018952D
:100028000C949206CFEFCDBFD4E0DEBFA09771D776
:10003800E3E0E0933001E0E0E0933101E0E2E093B7
:100048003201E5E0E0937C00E3ECE0937A00E0E045
:10005800E0937B005ED78CE07CD788E47AD72020B9
:10006800202020201F1FE6E6F0E0ABD781E071D703
:10007800E2E0F3D780E56DD72020201F1F20202045
:10008800E0E8F0E09ED781E064D7E2E0E6D788E5D3
:1000980060D72020201F1F201F1FEAE9F0E091D71A
:1000A80081E057D7E2E0D9D7E89430F81B9B02C02B
:1000B800689430F8EAE0E093B100E1EAE093B00038
:1000C8005B98539AE0E0E4BDE0E0E5BD5D985598A3
:1000D80030FE06C0EAE0E5BDE1EAE4BD5D98559A68
:1000E800E0E0E0938000E0E0E093810030FE04C0AF
:1000F800E0E4E7BDE7E0E8BDE0E4E093B300E4E076
:10010800E093B40030FE07C081E023D7E2E0A5D732
:10011800EAEFFEE03BD7E1E0AFD77894EEE7E09373
:100128000E01C7D5E0910801F0910901E0930A0199
:10013800F0930B01E0910801F0910901E09325018A
:10014800F093260180910E01E0910A018E1BE82FA1
:10015800E093220180E797E1E0912201FF27BDD7D4
:10016800E0931701F093180180910E019927E0910F
:100178000A01F0910B018E1B9F0BE82FF92FE093DA
:100188001501F09316018091150190911601EAE08E
:10019800F0E094D7E0931501F093160180911501D2
:1001A80090911601E0E1F0E098D7E0931501F09303
:1001B80016018FEB8F93E1E08F918E0FCAD6ECEF8B
:1001C800FEE0E4D6E0910A01F0910B0104D7D8D6FD
:1001D800E1E052D781E0BDD6E2E03FD7E8E7E0931F
:1001E8001401E0E0F0E0E0931101F0931201E894CB
:1001F80031F8E0E0E0932D01E0E0F0E0E093250144
:10020800F0932601E0E0E0931B01E0E0F0E0E093EA
:100218000C01F0930D01E0E0E0931C01E0E0E093B5
:100228001D01E0E0E0930401E0E0E0932E01E4EB3F
:10023800E0931301E0E0F0E0E0930F01F093100188
:10024800E89435F8E0912D01EF93E5E08F9129D7F7
:10025800E62FEF93E0E08F918E1709F04CC029D577
:100268008091080190910901E0910E01FF273196D4
:100278008E179F0708F407C0E0910E01FF27E0934F
:100288000801F09309018091080190910901E0911A
:100298000A01F0910B0131968E179F0708F411C0DF
:1002A8008091080190910901E0910A01F0910B01F8
:1002B8008E1B9F0BE82FF92FE0930801F09309019B
:1002C80006C0E0E0F0E0E0930801F09309018091B6
:1002D8000C0190910D01E0910801F0910901E80FDE
:1002E800F91FE0930C01F0930D0180912C01E1E0DE
:1002F800E80FE0932C0180912D01E0E08E1709F0C2
:10030800A9C030FE40C0E4E0E0937C00E3ECE09359
:100318007A00E4E0F0917C00F07EEF2BE0937C0023
:100328003DD6E0932301F0932401E0E0E0937A00C6
:100338008091230190912401E1E1F0E0CED6E09391
:100348002301F09324018091230190912401E4E09A
:10035800F0E0E80FF91FE0932301F0932401809166
:10036800230190912401EFE3F0E031968E179F0767
:1003780008F406C0EFE3F0E0E0932301F0932401D2
:10038800E0912301E8BDE5E0E0937C00E3ECE09335
:100398007A00E5E0F0917C00F07EEF2BE0937C00A2
:1003A800FDD5E0932301F0932401E0E0E0937A0087
:1003B8008091230190912401E0E1F0E08ED6E09352
:1003C8002301F09324018091230190912401EEE10F
:1003D800F0E031968E179F0708F406C0EFE1F0E0D1
:1003E800E0932301F0932401E0E0E093070180917A
:1003F800230190912401EEE1F0E08E179F0708F0A9
:1004080003C0E1E0E093070180912301909124016A
:10041800E0E0F0E08E179F0709F003C0E2E0E09308
:10042800070180910701E1E08E1709F403C0E0E0BD
:10043800E093040184E1E0912301E80FE0932701B0
:100448008AE0E0912301E80FE0932801E09123017D
:10045800E0932901E0912D01EF93EAE08F9121D6F5
:10046800E62FEF93E0E08F918E1709F0E6C28091B6
:100478000C0190910D01E0912C01FF272ED6E093FD
:100488000801F0930901E0910801F0910901FF9337
:10049800EF93EAE0F0E08F919F9110D6FF93EF93EE
:1004A800E0911501F09116018F919F9116D6E09376
:1004B8000C01F0930D018091110190911201E091CE
:1004C8001401FF2731968E179F0708F40DC0E0E04E
:1004D800F0E0E0931101F0931201E89431F8E0E0C4
:1004E800E0932E01E89435F8809108019091090174
:1004F800E5E0F0E031968E179F0708F419C0809167
:100508000F0190911001E0E0F0E08E179F0709F0CD
:1005180008C0689431F8E0E0F0E0E0931101F0934E
:100528001201E0911301FF27E0930F01F0931001EE
:1005380032FC9BC031FE15C080912E01E0E0E395AE
:100548008E1708F002C035FE0CC080911101909101
:100558001201E1E0F0E0E80FF91FE0931101F093D8
:1005680012018091080190910901E0911B01FF2778
:1005780031968E179F0708F404C0E0910801E093B4
:100588001B01E0910801F0910901FF93EF93E2E06C
:10059800F0E08F919F91E80FF91FFF93EF93E0919F
:1005A8001B01FF278F919F918E179F0708F04BC063
:1005B8008091020190910301EEE1F0E031968E17EF
:1005C8009F0708F404C0E8E2E0932F010DC0809172
:1005D8000201E2E05AD5E0932F0184E6E0912F0171
:1005E8008E1BE82FE0932F0131FE03C084E1809336
:1005F8002F01E0910801F0910901FF93EF93E09139
:100608002F01FF278F919F9159D5FF93EF93E4E630
:10061800F0E08F919F9161D5E0931901F0931A0151
:10062800689433F8E0911B01E0931D01689432F857
:10063800E0E0E093050131FE06C080912E01E1E083
:10064800E80FE0932E018091080190910901E09153
:100658001B01FF278E179F0708F007C0E0911B01B9
:10066800FF27E0930801F093090132FE2DC0809125
:10067800080190910901E0911B01FF278E179F0740
:1006880008F004C0E0910801E0931B01E091080123
:10069800F0910901FF93EF93E0911B01FF27FF936E
:1006A800EF93E2E0F0E08F919F91E80FF91F319608
:1006B8008F919F918E179F0708F406C0E89432F82F
:1006C800E0911B01E0931C0132FE44C080910801B7
:1006D80090910901E0911901F0911A0131968E1754
:1006E8009F0708F40DC080910701E1E08E1709F01B
:1006F80007C0E0911D01FF27E0930801F09309016D
:1007080080910401E0E0E3958E1708F423C08091FE
:100718000501E0E08E1709F01DC080910401E1E0B9
:100728008E1BE82FE093040180910401E0E0E3953B
:100738008E1708F409C0E0910401EF93E1E08F916E
:100748008E1BE82FE0930401E1E0E0930501E0E06F
:10075800E093060180910701E1E08E1709F028C0B7
:1007680032FC26C08091080190910901E09127018F
:10077800FF2731968E179F0708F41AC0809106014B
:10078800E0E08E1709F014C079D2809102019091AF
:100798000301EBE2F0E08E179F0708F009C085E03F
:1007A800E0910401E80FE0930401E1E0E093060121
:1007B80065D280910F0190911001E0E0F0E0319650
:1007C8008E179F0708F412C0E0910F01F0911001F5
:1007D800FF93EF93E1E0F0E08F919F918E1B9F0BC9
:1007E800E82FF92FE0930F01F093100180910F018A
:1007F80090911001E0E0F0E08E179F0709F00FC01C
:10080800E0E0E0930401E0E0E0930501E0E0E0933C
:100818000601E0E0E0931D0158D3E89431F8E8942C
:1008280034F8E0910801F0910901E0931E01F0937A
:100838001F01E0912301F0912401FF93EF93EAE077
:10084800F0E08F919F9149D4FF93EF93E1E0F0E0BE
:100858008F919F91E80FF91FE0930001F093010138
:1008680080910701E1E08E1709F06BC080910801C3
:1008780090910901E0910001F09101018E179F0705
:1008880008F002C031FE5DC031FE59C0E09102019E
:10089800F0910301FF93EF93E0911101F0911201A0
:1008A8008F919F910BD4FF93EF93E0911401FF2751
:1008B8008F919F9112D4E0930201F09303018091EC
:1008C800020190910301EAE0F0E08E179F0708F01B
:1008D80006C0EAE0F0E0E0930201F0930301E0E0F3
:1008E800F0E0E0930001F093010135FC28C080910D
:1008F800080190910901E0912801FF2731968E1790
:100908009F0708F41CC0689435F8809108019091FD
:100918000901E0912701FF2731968E179F0708F4F8
:1009280008C0E0912901EF93EFE08F91E80FE09381
:100938000401E8E7F0E0E0931101F09312016894F4
:1009480034F834FE36C08091080190910901E09195
:100958000001F09101018E1B9F0BE82FF92FE09306
:100968001E01F0931F0180911E0190911F01E091DB
:100978000201F0910301A2D3E0931E01F0931F013D
:1009880080911E0190911F01EAE0F0E0A6D3E09368
:100998001E01F0931F0180911E0190911F01E091AB
:1009A8000001F0910101E80FF91FE0931E01F09397
:1009B8001F0180911E0190911F01E0912201FF27E4
:1009C80031968E179F0708F407C0E0912201FF2790
:1009D800E0931E01F0931F0180912901EFE18E172A
:1009E80009F006C0E0E0F0E0E0932501F09326016D
:1009F800E0912501F0912601FF93EF93EAE0F0E002
:100A08008F919F915BD3FF93EF93E0911501F09144
:100A180016018F919F9161D3E0932001F0932101FA
:100A280080910701E2E08E1709F006C0E0E1F0E0EE
:100A3800E0932001F093210197D180910701E2E032
:100A48008E1709F40BC080911E0190911F01E4E6F6
:100A5800F0E031968E179F0708F446C0E091220116
:100A6800FF27FF93EF93E0912D01FF278F919F912F
:100A78008E1B9F0BE82FF92FFF93EF93EFE0F0E029
:100A88008F919F91E80FF91FE0931E01F0931F01CA
:100A980080912A01E9E08E1709F016C0E0910A0159
:100AA800F0910B01E0931E01F0931F01E0910A0100
:100AB800F0910B01E0930801F0930901E0E0F0E008
:100AC800E0932001F093210180912A01E5E08E173F
:100AD80009F009C08FE78F93E1E08F918E0F39D22B
:100AE800E0E0FFE053D203C0E0E0E0932A01809108
:100AF8001E0190911F01E4E6F0E08E179F0708F0B1
:100B080044C0E0912501F0912601FF93EF93E09115
:100B18001E01F0911F01FF93EF93E1E0F0E08F9148
:100B28009F91E80FF91F31968F919F918E179F071C
:100B380008F412C0E0912501F0912601FF93EF938C
:100B4800E1E0F0E08F919F918E1B9F0BE82FF92F2A
:100B5800E0932501F09326018091250190912601CB
:100B6800E0911E01F0911F018E179F0708F00CC03D
:100B78008091250190912601E1E0F0E0E80FF91F4E
:100B8800E0932501F093260108C0E0911E01F09141
:100B98001F01E0932501F0932601E0912501F091D2
:100BA8002601FF93EF93E0911701F09118018F91BF
:100BB8009F9184D2FF93EF93E4E6F0E08F919F91A9
:100BC8008CD2FF93EF93E4E0F0E08F919F91E80FD0
:100BD800F91FE0930001F0930101809100019091C9
:100BE8000101EFE3F0E031968E179F0708F406C085
:100BF800EFE3F0E0E0930001F09301018091290117
:100C0800EFE18E1709F006C0E4E0F0E0E0930001A0
:100C1800F0930101E0910001E093B40080912D016F
:100C2800E1E0E80FE0932D0180912D01EFE18E17AF
:100C380009F023C0E0E0E0932D0180910701E2E094
:100C48008E1709F40BC080911E0190911F01E4E6F4
:100C5800F0E031968E179F0708F40FC080912A01A3
:100C6800E1E0E80FE0932A0180912A01EAE08E177B
:100C780009F003C0E0E0E0932A01E4CAE8E2F0E00A
:100C8800FF93EF93E0912901FF278F919F918E1B8E
:100C98009F0BE82FF92FFF93EF93E0910401FF27B3
:100CA8008F919F91E80FF91FE0930201F0930301E0
:100CB8000895E0E0E0938700E0E0E0938600E0E25A
:100CC800E0936F00E2E0D2D1E2E4E093810080910A
:100CD8008600E0E08E1709F006C0E0E0F0E0E0935F
:100CE8000801F0930901E0E4C1D1E0E0E0936F006E
:100CF800E2E0BCD18091080190910901E091840063
:100D0800FF278E179F0709F408C0E0918400FF278A
:100D1800E0930801F0930901CCCF08952FB6EF9323
:100D2800FF930F921F928F939F93AF93BF938091DE
:100D38008100E2E48E1709F00AC0E2E0E093810046
:100D4800E0E0E0938500E0E0E093840003C0E0E0A9
:100D5800E0938100BF91AF919F918F911F900F9069
:100D6800FF91EF912FBE1895E1E0E0932C01E0E1AF
:100D78005F92E3955E2E8FEB8F93E0912C018F911C
:100D88008E0FE7D0E0E0E0932B0180910C01909169
:100D98000D01E0912C01FF278E179F0708F408C06A
:100DA800E0912B01EF93E2E08F91E80FE0932B01A4
:100DB8008091200190912101E0912C01FF278E174D
:100DC8009F0708F408C0E0912B01EF93E1E08F91B1
:100DD800E80FE0932B0180912B01E0E0E3958E175B
:100DE80008F405C0E0912B018E2FB1D003C0E6E0D6
:100DF800FFE0CCD0E0912C01E395E0932C01E515C0
:100E080008F4B9CF5F90E0E0E0932C01E0E0F0E077
:100E1800E0930C01F0930D01E2E0E0933001E0E093
:100E2800E093310133FE01C050D08FE78F93E1E0AA
:100E38008F918E0F8ED0E1E0E0933001E1E0E093F6
:100E4800310180910701E2E08E1709F004C0E8E063
:100E5800FFE09CD039C080912901EFE18E1708F09E
:100E680030C080910401E0E0E3958E1708F40DC0CE
:100E7800EEE0FFE08BD0E0910201F0910301ABD0EE
:100E88007FD0E6E0FFE082D01BC031FC0DC0E0E17E
:100E9800FFE07CD0E0910201F09103019CD070D07A
:100EA800E6E0FFE073D00CC0E2E1FFE06FD0E09134
:100EB8000201F09103018FD063D0E6E0FFE066D035
:100EC80003C0E4E1FFE062D00895E2E0E09330017E
:100ED800E0E0E0933101E89433F88FE78F93EFE097
:100EE8008F918E0F36D0E0911D0173D049D00895AF
:100EF800FFCF440054513D00202020202000200036
:100F08002D4D41582D004100780053003D4F464675
:100F18003D00E7B1EF60E7B9509A519A589859984F
:100F2800E8E19BD083E01AD0E8E097D01ED0EDE04E
:100F38009DD01BD0409819D088E20BD086E009D00C
:100F48008CE007D081E005D0E4E087D00895589A76
:100F580001C05898582F829501D0852F78B1707F9D
:100F68008F70872B88B901D00895599A0000000026
:100F7800000000005998EF93E4E078D0EF910895CD
:100F88008191882311F0E3DFFBCF0895C89531964E
:100F9800002019F0802DDBDFF9CF0895E0917A0069
:100FA800E660E0937A00E0917A00E4FFFCCF80915C
:100FB8007A00846080937A00E0917800F09179005B
:100FC800089598E0C8953196802DC1DF9A95D1F79C
:100FD8000895FF27E894E89408C0E894F7FF05C04F
:100FE800E095F095EF5FFF4F6894CF93DF936F9292
:100FF8009091310166246A92992319F015D06EE216
:101008006A939091300110D0992329F060913201B0
:101018006A939A95E9F716F4EDE2EA93EC2F6F904C
:10102800FD2FDF91CF91089550E1661B6694EE1F66
:10103800FF1F661F661C6A3010F06A40E3955A95D8
:10104800A9F7605D6A939A9519F06E2F6F2B09F4D2
:1010580008956E2F6F2B41F7089544E155E85A958E
:10106800F1F74A95D9F7EA95C1F7089569E16A95C4
:10107800F1F7EA95D9F70895FE2F64E0EAEFEDDF7E
:101088006A95E1F7FA95C9F70895FF93FF2738E0C5
:10109800E69508F4F80FF795E7953A95D1F7FF919B
:1010A8000895661B79E004C0661F6E1708F06E1B72
:1010B800881F7A95C9F78095E82F089577276627BE
:1010C80050E1F695E79510F4680F791F77956795C5
:1010D800F795E7955A95B9F708956E2F7F2FE82F62
:1010E800F92F8827991B41E1EE1FFF1F4A9509F444
:1010F8000895881F991F861B970B20F4860F971F4A
:081108008894F2CF0894F0CFA7
:00000001FF
